:1000000010308500831603138501811383120313B7
:1000100010308500831603138111811201118312A0
:100020000313940196017A30970081010B110B1D87
:1000300017280B1106088F009001910192012220D0
:100040007D2017280030140203193E2801301402C5
:1000500003194328023014020319482803301402FC
:1000600003194D28043014020319522805301402D4
:1000700003195728950B080094010800AA30930033
:100080005D20940A08000F0893075D20940A080079
:10009000100893075D20940A0800110893075D205B
:1000A000940A0800120893075D20940A08001308B8
:1000B0005D200A309500940A08008D0005121F305B
:1000C0008C008C0B6128642808308E008D0C03187E
:1000D0006C28000005126E2805166E281F308C0053
:1000E0008C0B70288E0B6628752876280000051664
:1000F00045308C008C0B7A2808000030160203195A
:1001000088280510970B08007A309700960308009E
:0E0110000514970B08007A309700960A080035
:02400E00F11FA0
:00000001FF
